:060000000A128A11122809
:10000800FE00030EF1000408F2000A08F300831250
:1000180003137F08F4000A128A117B2D0A128A1131
:100028001528F601F701F801F901FA0183132030C8
:10003800840056300A128A15C72583010A128A11CC
:1000480025288B01831203139F010630831603139F
:100058009F003F3083120313850009308316031372
:1000680085000630831203138600063083160313B7
:100078008600903083120313870090308316031391
:1000880087008430810083120313B2017D30EC00B5
:100098006C08EE00B1017B14FA01B0010030D60003
:1000A8000030D7000930D8000030D9004D300A128E
:1000B8008A11DE270A128A1183120313B701B801C5
:1000C800B601B401B501B301A001A101A301A401C6
:1000D800A201A801A901AB01AC01AA01A501F8017F
:1000E800F701A701A601F901AE01F6117611AF01DA
:1000F8000030D6000030D7001430D8000030D900C6
:1001080039300A128A11DE270A128A11F61076127D
:1001180083120313AD017610871276150A128A1519
:10012800E2250A128A1106308312031381008B1606
:100138000B17831603138C160A128A110A260A1241
:100148008A110A128A1154260A128A110A128A1569
:10015800C1250A128A118B177A08023A031DBF2893
:10016800831203133008013A031DBF280A128A15A7
:1001780013260A128A117A08043A031DCE2883121C
:1001880003133008013A031DCE280A128A111124DC
:100198000A128A117A08063A031DDD28831203130E
:1001A8003008013A031DDD280A128A15F6250A12BD
:1001B8008A117A08083A031DEC28831203133008C1
:1001C800013A031DEC280A128A11C6240A128A1160
:1001D8007A080A3A031DFB28831203133008013AF0
:1001E800031DFB280A128A1175220A128A117A083D
:1001F8000C3A031D0A29831203133008013A031D20
:100208000A290A128A15BC250A128A117A080E3A96
:10021800031D1929831203133008013A031D1929F4
:100228000A128A1148230A128A11F908031D1F2984
:1002380083120313AF011430831203132F02031C1C
:100248006A297611F611AF0183160313A001A101E3
:1002580013302102031859292108393E84008313D9
:10026800000883120313EC006C08D60083160313EE
:100278002108013E0A128A15CF250A128A1183160F
:100288000313200783120313ED006D08831603136D
:10029800A000013083120313EC006C0883160313CB
:1002A800A10713302102031C3029831203134C08C1
:1002B800831603132006031D6929831203133908C3
:1002C800093A031D6929F6146A297615F61C5D2A70
:1002D800F61083123B08C13A031D7729C230EC009F
:1002E8006C08BB0076163B08013A031D80293208CA
:1002F800EC006C08BC0076163B08023A031DC529C1
:100308003708EC006C08BC003808EC006C08BD002D
:100318003608EC006C08BE003408EC006C08BF001E
:100328003508EC006C08C0003308EC006C08C1000C
:100338002008EC006C08C2002108EC006C08C3001F
:100348002308EC006C08C4002408EC006C08C50005
:100358002208EC006C08C6002808EC006C08C700EE
:100368002908EC006C08C8002B08EC006C08C900D0
:100378002C08EC006C08CA002A08EC006C08CB00BA
:100388007616761E5A2A76123A08EC006C08B900DE
:100398000930EC006C08BA0083160313A001A10110
:1003A800133021020318012A2108393E84008313DF
:1003B800000883120313EC006C08D600831603139D
:1003C8002108013E0A128A15CF250A128A118316BE
:1003D8000313200783120313ED006D08831603131C
:1003E800A000013083120313EC006C08831603137A
:1003F800A10713302102031CD829200883120313F4
:10040800EC006C08CC000A30EC006C08831603136F
:10041800A000212AA0080319242AF6110D308312FE
:100428000313ED00FB30EC00EC0B182AED0B182A37
:100438001D2A013083160313A002F6190E2A76141A
:10044800761C5A2A7610043083120313EC006C08C9
:10045800AE00871683160313A10114302102031876
:10046800572A2108393E8400831300088312031396
:1004780099000230EC006C08F900831603139818F1
:10048800482AF908031D412AF9080319572A013097
:1004980083120313EC006C0883160313A1071430AE
:1004A8002102031C352A8312031387128312AF011A
:1004B800761577088312270603196C2A7708013AFC
:1004C800031D682A0130FB067708EC006C08A700BA
:1004D8007B1C702A3216B028EF30EC006C08B2058D
:1004E800B0280A128A119E260A128A110038031DA2
:1004F800842AFB3083120313DE005E08B20508006D
:100508000A128A11E2260A128A1183120313DE00E4
:100518005E08E9000A128A11E2260A128A11831279
:100528000313DE005E08E8000A128A11E2260A12A6
:100538008A1183120313DE005E08EB000A128A1187
:10054800E2260A128A1183120313DE005E08EA000B
:100558000A128A11E2260A128A1183120313DE0094
:100568005E08E20068086907DE006B085E07DF00C6
:100578006A085F07E0006008E30062086306031981
:10058800CA2AFB30DE005E08B2050800EB1FD42A39
:100598006B087F39DE005E08EB00A201A20AD52AAB
:1005A800A2016808DE00DF016908E000E1016008D7
:1005B800E100E0015E086004E4005F086104E50012
:1005C8006A08DE00DF016B08E000E1016008E10075
:1005D800E0015E086004E6005F086104E7000A3095
:1005E800D6000030D7006508D901D9076408D801BA
:1005F800D8070A128A1124270A128A1183120313B0
:100608005608DE005E08A0000A30D6000030D70089
:100618006508D901D9076408D801D8070A128A15CC
:10062800E0260A128A11831203135608DE005E08B8
:10063800A1000A30D6000030D7006708D901D907D1
:100648006608D801D8070A128A1124270A128A11C3
:10065800831203135608DE005E08A3000A30D60092
:100668000030D7006708D901D9076608D801D8072C
:100678000A128A15E026831203135608DE005E0864
:10068800A400B0013215080083120313051C0A2CBC
:100698000A128A15AD260A128A1183120313DE0084
:1006A8005E08E2000A128A15AD260A128A11831220
:1006B8000313DE005E08E3000A128A15AD260A124B
:1006C8008A1183120313DE005E08E4000A128A15F9
:1006D800AD260A128A1183120313DE005E08E500B4
:1006E8006308DE00DF016208E000E1016008E10064
:1006F800E0015E086004E8005F086104E900033077
:100708006902E8300319680203189C2B6809DE00A7
:100718006909DF00DE0A0319DF0A5E08E83EE8001F
:100728005F080318013E033EE900AA01AA0AA52BA7
:100738006808183EE80069080318013EFC3EE90015
:10074800AA010A30D6000030D7006908D901D907B4
:100758006808D801D8070A128A1124270A128A11B0
:10076800831203135608DE005E08AB000A30D60079
:100778000030D7006908D901D9076808D801D80717
:100788000A128A15E0260A128A11831203135608E0
:10079800DE005E08AC006508DE00DF016408E000EA
:1007A800E1016008E100E0015E086004E6005F081E
:1007B8006104E7006430D6000030D7006708D9012B
:1007C800D9076608D801D8070A128A1124270A12FD
:1007D8008A11831203135608DE005E08A8006430ED
:1007E800D6000030D7006708D901D9076608D801B4
:1007F800D8070A128A15E0260A128A1183120313EF
:100808005608DE005E08A900B2150E2CF730DE008F
:100818005E08B2050511B00108000A128A15812682
:100828000A128A110038031D202CFE30831203138C
:10083800DE005E08B2050800CC300A128A154E2781
:100848000A128A11BE300A128A154E270A128A1114
:1008580083120313E201093062020318492C0A12B9
:100868008A11A1270A128A1183120313DE00620873
:100878004D3E84005E08831380000130DE005E0870
:10088800E20709306202031C332C0A128A1164271A
:100898000A128A110318572CFE3083120313DE0044
:1008A8005E08B2050800831203134D08DE00DF015D
:1008B8004E08E000E1016008E100E0015E08600424
:1008C800E3005F086104E4006408DF006308DE00F9
:1008D80004300310DF0CDE0CFF3E031D6D2C5E0898
:1008E800E3005F08E400E41D812CE309E409E30A5E
:1008F8000319E40AB601B60A822CB6016308DE00C1
:100908005E08B700E301E40163084D04E3006408EE
:10091800E4000F306305E30000306405E400640878
:10092800D701D7076308D601D6077130D80002303F
:10093800D9000A128A1530260A128A118312031363
:100948005708E401E4075608E301E307E830D60056
:100958000330D7006408D901D9076308D801D8073C
:100968000A128A112427831203135708E401E407A3
:100978005608E301E3076308DE005E08B800B0012B
:10098800321408000A128A1555260A128A110038EC
:10099800031DD52CFD3083120313DE005E08B2055B
:1009A8000800CC300A128A1516270A128A11BE309E
:1009B8000A128A1516270A128A1183120313E201F2
:1009C800093062020318FE2C0A128A1586270A12B9
:1009D8008A1183120313DE0062084D3E84005E080C
:1009E800831380000130DE005E08E20709306202EE
:1009F800031CE82C0A128A15C3270A128A11031845
:100A08000C2DFD3083120313DE005E08B2050800CA
:100A1800831203134D08DE00DF014E08E000E101F8
:100A28006008E100E0015E086004E3005F0861041B
:100A3800E4006408DF006308DE0004300310DF0C04
:100A4800DE0CFF3E031D222D5E08E3005F08E40074
:100A5800E41D362DE309E409E30A0319E40AB301A6
:100A6800B30A372DB3016308DE005E08B400E30162
:100A7800E40163084D04E3006408E4000F306305F3
:100A8800E30000306405E4006408D701D707630871
:100A9800D601D6077130D8000230D9000A128A155B
:100AA80030260A128A11831203135708E401E40757
:100AB8005608E301E307E830D6000330D70064089E
:100AC800D901D9076308D801D8070A128A1124273F
:100AD800831203135708E401E4075608E301E30708
:100AE8006308DE005E08B500B001B21408000B1DF3
:100AF800D22D0B11063081000130EE02EE08031DE5
:100B0800972D7D30F0007008EE000430F00070087A
:100B1800B1000130F0007008FA07B001B00A1430D3
:100B28007A020318FA0131080319A02D0130B10225
:100B38007B1CA12D8715A12D87112E080319AA2D1D
:100B48000130AE027B1CAB2D0715AB2D07117908C0
:100B58000319B02D0130F90225080319B52D01300C
:100B6800A502A508031DD22DF801071ABD2DF8010D
:100B7800F80A78082606031DC62D7808F0007008C4
:100B8800F700D22D7808F0007008A600F701770862
:100B98000319D22D0630F0007008A5008C1EFF2D19
:100BA8000230F0007008F9008C129818DD2D181D1D
:100BB800E82D981CE12D18121816181DFF2D1A087B
:100BC800F0007008F500FF2DF6151A08F0007008FF
:100BD800F500761DFF2D14302F020318FF2D750820
:100BE800F0002F08393E840070088313800001301C
:100BF800F0007008AF077408FF0073088A007208D5
:100C08008400710E8300FE0E7E0E09000A128A15FA
:100C180081260A128A110038031D192EFE3083120C
:100C28000313DB005B08B2050800CC300A128A15F2
:100C38004E270A128A114E300A128A154E270A12B6
:100C48008A117D300A128A154E270A128A11C93074
:100C58000A128A154E270A128A1160300A128A155A
:100C68004E270A128A110A128A1581260A128A1137
:100C78000038031D462EFE3083120313DB005B0889
:100C8800B2050800CC300A128A154E270A128A11BA
:100C980048300A128A154E2783120313B001080040
:100CA8000A128A1555260A128A110038031D632E66
:100CB800FD3083120313DB005B08B2050800CC305B
:100CC8000A128A1516270A128A114E300A128A1534
:100CD80016270A128A117D300A128A1516270A1257
:100CE8008A11C9300A128A1516270A128A11603029
:100CF8000A128A1516270A128A110A128A15552607
:100D08000A128A110038031D902EFD308312031336
:100D1800DB005B08B2050800CC300A128A151627DA
:100D28000A128A1148300A128A15162783120313E9
:100D3800B001080083120313D7018316031386102A
:100D4800831203138610F930D6000000D60BA92EA3
:100D5800AD2E000083160313861483120313861422
:100D68008618B82E570808006430D6005608D800F0
:100D7800C22ED8080319C42E0130D8028618BD2EF9
:100D88008618C82ED701D70A6430D6005608D8006E
:100D9800CF2E0130D8028618D42ED808031DCD2EA8
:100DA8006430D6005608D800DB2E0130D802861CE5
:100DB800E02ED808031DD92E570808008312031304
:100DC800DA01D801D80A093058020318222F6430F2
:100DD800D6005608D900F22E0130D9028618F72E0F
:100DE800D908031DF02E0B30D600D60BF92E0000C3
:100DF800831203135A08D6005607D7005708DA009B
:100E0800861C092F5A0801380B2F5A08FE39D600BC
:100E18005608DA006430D6005608D900152F01307C
:100E2800D902861C1A2FD908031D132F0130D600AA
:100E38005608D80709305802031CEB2E5A08080038
:100E480083120313DC01DD015708560403195D2FD3
:100E5800DB01DB0AD71B3C2F01300310D60DD70D61
:100E6800FF3E031D312F0130DA005A08DB072E2F11
:100E780001300310DC0DDD0DFF3E031D3D2F57082B
:100E88005902031D492F56085802031C522F5608B1
:100E9800D8025708031CD903D9025C140130031087
:100EA800D70CD60CFF3E031D532F0130DB02031D68
:100EB8003C2F5D08D701D7075C08D601D607080084
:100EC80083120313DA01D901083059020318992F44
:100ED80059084D3E8400831300085A06D600560868
:100EE800DA00D801083058020318912F5A1C822FB3
:100EF8005A08D6000310560C8C3A862F5A08D6008A
:100F08000310560CD7005708DA000130D6005608EF
:100F1800D80708305802031C7A2F0130D60056082B
:100F2800D90708305902031C6C2F55085A06031DAF
:100F38009F2F031408000310080083120313D9011C
:100F4800D801D80A093058020318DC2F8316031376
:100F58008511831203138511B12F83160313851589
:100F68008312031385150330D600D60BB92F8312CD
:100F780003135908D6000310560CD7005708D90098
:100F8800851DC92F59088038CB2F59087F39D600BD
:100F98005608D9002130D600D60BD02F0130831245
:100FA8000313D6005608D80709305802031CAA2F85
:100FB8005908080083120313DC005C08DA005A0899
:100FC800DB000130D8020030031CD903D902FF30FE
:100FD8005906031DF12FFF3058060319080056085B
:100FE800DA005B0884005A08831380000130DA00B5
:060FF8005A08DB07E52F9B
:101B7800831203130515B00108008312031305111E
:101B88008514B001080064008001840A0406031962
:101B980000340406C82D83120313D900D801591C38
:101BA800D92D5608D7005708D8070310D60D0310AB
:101BB800D90CD908031DD32D580808008316031320
:101BC80018150C309900181283120313981718135C
:101BD800831603131813831203131816831603139B
:101BE800981608000A128A1555260A128A1500380E
:101BF800031D052EFD3083120313DB005B08B205BD
:101C08000800CC300A128A1516270A128A154430A1
:101C18000A128A15162783120313B00108000A1244
:101C28008A1581260A128A150038031D222EFE30D5
:101C380083120313DB005B08B2050800CC300A12DC
:101C48008A154E270A128A1544300A128A154E2719
:101C580083120313B001080083120313DA01DB01B6
:101C6800561C3C2E5808DA070318DB0A5908DB070C
:101C780001300310D80DD90DFF3E031D3D2E013054
:101C88000310D70CD60CFF3E031D442E57085604EC
:101C9800031D342E5B08D701D7075A08D601D6078B
:101CA800080083120313D701831603130611831246
:101CB80003130611A630D600D60B602E000083163B
:101CC8000313061583120313061506196D2E00302B
:101CD80008001530D600D60B6F2E000083120313B0
:101CE8000619782ED701D70A4F30D600D60B7A2E90
:101CF8007D2E831203135708080083120313D7019C
:101D0800831603138511831203138511A630D60099
:101D1800D60B8C2E0000831603138515831203132C
:101D280085158519992E003008001530D600D60B78
:101D38009B2E0000831203138519A42ED701D70AFE
:101D48004F30D600D60BA62EA92E831203135708A0
:101D5800080083120313D901D801D80A09305802A0
:101D68000318DE2E85101830D600D60BB92EBC2EDF
:101D78008312031385145908D6005607D70057084D
:101D8800D900051CCA2E59080138CC2E5908FE392D
:101D9800D6005608D9001830D600D60BD12ED42E2E
:101DA800013083120313D6005608D80709305802A9
:101DB800031CB62E5908080083120313570856044B
:101DC80003190F2FDB01DB0AD71BF62E0130031096
:101DD800D60DD70DFF3E031DEB2E0130DA005A0851
:101DE800DB07E82E57085902031DFC2E5608580237
:101DF800031C042F5608D8025708031CD903D9021C
:101E080001300310D70CD60CFF3E031D052F0130FF
:101E1800DB02031DF62E5908D701D7075808D6014B
:101E2800D607080083120313D8005808D6005608AE
:101E3800DA00D901D90A09305902031808008316B3
:101E4800031306118312031306112A2F8312031397
:101E58005A1C342F83160313061583120313061511
:101E68005A08D6000310560CD7005708DA0013306A
:101E7800D600D60B3D2F402F831603130615831269
:101E880003130615472F013083120313D600560893
:101E9800D9071F2F83120313D8005808D6005608F5
:101EA800DA00D901D90A0930590203180800831643
:101EB80003138511831203138511622F83120313F1
:101EC8005A1C6C2F8316031385158312031385156B
:101ED8005A08D6000310560CD7005708DA001330FA
:101EE800D600D60B752F782F83160313851583120A
:101EF800031385157F2F013083120313D60056086C
:101F0800D907572F83120313D901D801D80A0930EA
:101F180058020318C12F83160313061183120313E3
:101F28000611962F8316031306158312031306153D
:101F38000330D600D60B9E2F831203135908D60000
:101F48000310560CD7005708D900061DAE2F5908A4
:101F58008038B02F59087F39D6005608D90021306B
:101F6800D600D60BB52F013083120313D6005608BE
:101F7800D80709305802031C8F2F5908080083120C
:101F88000313DA01D901083059020318F82F590848
:101F98004D3E8400831300085A06D6005608DA001E
:101FA800D801083058020318F02F5A1CE12F5A089C
:101FB800D6000310560C8C3AE52F5A08D6000310A9
:101FC800560CD7005708DA000130D6005608D80753
:101FD80008305802031CD92F0130D6005608D907FB
:101FE80008305902031CCB2F55085A06031DFE2F33
:081FF8000314080003100800A7
:02400E0071FF40
:00000001FF
